:020000040000FA
:10000000C0230020150200001D0200001F02000096
:100010002102000023020000250200000000000071
:1000200000000000000000000000000027020000A7
:1000300029020000000000002B0200002D02000039
:100040002F0200001D0300002F0200002F020000FD
:100050002F0200002F0200002F0200002F020000DC
:100060002F0200002F0200002F0200002F020000CC
:100070002F0200002F0200002F0200002F020000BC
:100080002F0200002F0200002F0200002F020000AC
:10009000790300002F0200002F0200002F02000051
:1000A0002F0200002F020000ED0600002F020000CA
:1000B0002F0200002F0200000000000000000000DE
:1000C0002F0200002F0200002F0200002F0200006C
:1000D0002F0200002F0200002F020000000000008D
:1000E0000000000000000000000000000000000010
:1000F0000000000000000000000000000000000000
:1001000000000000000000000000000000000000EF
:1001100000000000000000000000000000000000DF
:1001200000000000000000000000000000000000CF
:1001300000000000000000000000000000000000BF
:1001400000000000000000000000000000000000AF
:10015000000000000000000000000000000000009F
:10016000000000000000000000000000000000008F
:10017000000000000000000000000000000000007F
:10018000000000000000000000000000000000006F
:10019000000000000000000000000000000000005F
:1001A000000000000000000000000000000000004F
:1001B000000000000000000000000000000000003F
:1001C000000000000000000000000000000000002F
:1001D000000000000000000000000000000000001F
:1001E000000000000000000000000000000000000F
:1001F00000000000000000000000000000000000FF
:10020000DFF80CD000F03CF800480047F908000087
:10021000C02300200648804706480047FEE7FEE767
:10022000FEE7FEE7FEE7FEE7FEE7FEE7FEE7FEE7A6
:10023000D10300000102000040EA01039B0703D044
:1002400009E008C9121F08C0042AFAD203E011F815
:10025000013B00F8013B521EF9D27047D2B201E0D7
:1002600000F8012B491EFBD270470022F6E710B5BB
:1002700013460A4604461946FFF7F0FF204610BD14
:10028000064C074D06E0E06840F0010394E80700E3
:1002900098471034AC42F6D3FFF7B6FFF8140000CD
:1002A0001815000000F01F02012191404009800054
:1002B00000F1E020C0F88012704700F01F02012119
:1002C00091404009800000F1E020C0F880117047A3
:1002D00000F01F02012191404009800000F1E02060
:1002E000C0F80011704700F01F0201219140400941
:1002F000800000F1E020C0F8001270474907090EA5
:10030000002806DA00F00F0000F1E02080F8141D4C
:10031000704700F1E02080F80014704770B5144C6D
:10032000D4F80001002628B1D4F80403C00701D096
:10033000C4F80061D4F80C010E4D40B1D4F80403A8
:10034000000704D5C4F80C61286900B18047D4F8CF
:10035000100100280BD0D4F80403C00607D5C4F858
:100360001061E868002802D0BDE87040004770BD09
:1003700000100040280000207CB5144C606A0190F9
:100380002078002821D00120FFF797FF656800261C
:1003900066600120FFF79CFFE169002915D0E8079E
:1003A00003D08DF8006068468847A80705D501206E
:1003B0008DF80000E16968468847680705D5022086
:1003C0008DF80000E169684688477CBD2800002060
:1003D000F0B5B5480023021D0178101D01254FF02E
:1003E000805406290BD11678360708D10678C6F353
:1003F0000316032E06D0042E04D0052E02D00629A3
:1004000007D00EE0B4F82463A84FC6F304263E607C
:1004100002E01678360704D10678C6F30316032ED9
:1004200002D0062904D00FE0A24FA14E7E670EE055
:100430001678360708D10678C6F30316032E06D0C1
:10044000042E04D0052E02D0062907D00EE0D4F8E1
:100450004462994FC6F342363E6002E01678360792
:1004600004D10678C6F30316032E02D0062906D05F
:1004700011E0924E376827F0807737600EE01678EB
:10048000360708D10678C6F30316032E06D0042ECD
:1004900004D0052E02D006290AD011E04FF0804684
:1004A000C6F80C31C6F81031834E361F336002E0B7
:1004B0001678360704D10678C6F30316032E02D049
:1004C000062905D00CE07C4F032664373E600AE025
:1004D0001678360704D10678C6F30316032E02D029
:1004E00006290DD014E0764F05263E60744E78360E
:1004F0003560734E083633603F263F1D3E6002E094
:100500001678360704D10678C6F30316052E02D0F6
:10051000062957D062E06B4E36686B4F3E60694EDD
:10052000361D36683F1D3E60664E083636683F1DF4
:100530003E60644E0C3636683F1D3E60614E10369C
:1005400036683F1D3E605F4E143636683F1D3E6084
:100550005C4E183636685C4F20373E60594E1C366C
:1005600036683F1D3E60574E203636683F1D3E6060
:10057000544E243636683F1D3E60524E283636684B
:100580003F1D3E604F4E2C3636683F1D3E604D4E3F
:10059000303636684C4F40373E604A4E3436366807
:1005A0003F1D3E60474E383636683F1D3E60454E23
:1005B0003C3636683F1D3E60424E403636683F1D31
:1005C0003E6002E01678360708D10678C6F30316B7
:1005D000032E06D0042E04D0052E02D0062907D003
:1005E00019E0D4F85812394A01F04F01116002E0C5
:1005F000117809070FD10078C0F30310032803D046
:10060000042801D0052806D131480168C90702D065
:100610006FF001010160D4F83001062808D1D4F848
:100620003401062804D12B48016841F4806101603F
:1006300022487438016841F470010160BFF34F8FA4
:10064000BFF36F8F4FF01021D1F80002002803DBB9
:10065000D1F80402002822DA1F4A15601F480468F6
:10066000002CFCD01524C1F800420568002DFCD0F8
:10067000C1F8044201680029FCD013600168002918
:10068000FCD0BFF34F8F0D48F0380168144A01F4D5
:10069000E06111430160BFF34F8F00BFFDE71249D6
:1006A00010480860F0BD0000E00F00F04035014048
:1006B0000DF0ADBA00C007403C050040FCED00E085
:1006C000105600400404001020C50040E40E004015
:1006D000000400403C17004004E5014000E40140F4
:1006E0000400FA050090D003700000200748D0F8FD
:1006F0004011002909D00021C0F840110448407879
:10070000032802D1034901200861704700A001407D
:10071000280000200010004002E008C8121F08C195
:10072000002AFAD170477047002001E001C1121F72
:10073000002AFBD17047006890FAA0F000BA00BA16
:100740007047000072B609480068C00700D000BEBC
:10075000BFF34F8F0548E4380168054A01F4E061B2
:1007600011430160BFF34F8F00BFFDE7F0ED00E0E4
:100770000400FA050EB500210091CDE901106A468A
:1007800044F20100FFF7DEFF0EBD000006480168DD
:1007900021F0010101600548016821F0010141F0EB
:1007A00080710160002070475016004074170040AF
:1007B0002DE9FC410646C0074FF000050ED0104F52
:1007C00000240122385D009500231146019500F0B8
:1007D0009DFB641C042CF4D300F01CF8B0070DD56D
:1007E000074E0024361D0022305D0323009511467C
:1007F000019500F08BFB641C042CF4D3BDE8FC8154
:10080000F01400000249085C012100F09CBB0000CC
:10081000F014000010B500242046FFF7F3FF641C1D
:10082000042CF9D310BD006890FAA0F000BA70470C
:100830004FF080400021C0F800110121C0F80010E5
:10084000D0F800110029FBD07047000000B51BA0B4
:100850008BB0006808901AA01AA100680990D1E92D
:100860000001CDE90601182218496846FFF7E4FCAB
:1008700001208DF800008DF8080015480190002037
:100880008DF801004FF416718DF81400ADF80C10BE
:10089000684600F0DFF800280DD108A800F014FA2F
:1008A000002808D109A800F03DFA002803D108214A
:1008B00006A800F07DFA0BB000BD0000E7E7E7E70F
:1008C000C2C2C2C2E7C2C3C4C5C6C7C8D8140000EA
:1008D000E109000030B408200F214FF0A0430322AB
:1008E00003EB8004C4F80027401C8842F8D930BCD0
:1008F0000120FFF75DBF0000FFF7ECFFFFF798FF57
:10090000FFF7A4FF08B1FFF735FF214C214D224E20
:100910000027E7701E4800F0A3FAA0BBA0794107AA
:1009200003D000F00700042801D9012100E00021D4
:10093000112000F0FDFAA07900F00700012801D98C
:10094000052801D9012100E00021122000F0F0FA71
:10095000A07900F00700022801D9062801D9012159
:1009600000E00021132000F0E3FAA07900F0070076
:10097000032801D8012100E00021142000F0D8FA5A
:10098000A079401CA071691C30468847C1E700006F
:1009900000000020D014000000D4300070B50C49D5
:1009A0004FF4705008600B4C0025657000F0CEFBD2
:1009B00020210948FFF759FCE56214202563FFF761
:1009C0007CFC06490320C1F80002002070BD000035
:1009D00008F5014028000020A0030020001000407E
:1009E00010B50446007870B1012802D002280AD15F
:1009F00004E000F017F800F01FFA04E0074800F0E8
:100A00001FF90028FAD006494FF470400860207999
:100A10000007000C091F086010BD000074000020D2
:100A20000C050050094810B5007860B10120FFF7AF
:100A300044FC074800218162016241620120FFF706
:100A400047FC002010BD082010BD00002800002039
:100A5000DC0100202DE9F04105007DD0694C2078B3
:100A600018B1FFF79BFF002877D16868E061182272
:100A700029466548FFF7E0FB0025656020216348B3
:100A8000FFF7F3FBE562256300F0A4FC00287DD0AE
:100A90005F494FF0E7300860091D4FF043300860B0
:100AA000091D5C480860091D5B48086000F04EFBAA
:100AB00055490020183101F5947200BF00EB800306
:100AC00003EB40130B4442F82030401C0828F5DBB0
:100AD0005249002001F5947200EB800303EB4013B0
:100AE0000B4442F82030401C0828F5DB4C48042613
:100AF00006604B48083805604A4840F20221C0F8B9
:100B000000124A4A48491160111D0860DFF8188137
:100B1000091D08F10408C1F80080001D091D0860C6
:100B2000091D434808604048F038091D08604048E6
:100B3000001D091D0860091D3E480860324F787C81
:100B400000F007010120FFF7D9FBB87C00F0070196
:100B50001420FFF7D3FB01E04FE04CE01420FFF737
:100B6000B7FBA0780127E8B3A068294940F040000E
:100B7000A0600220443108602F49032008602E48FD
:100B8000083006602C490520383100E037E0086065
:100B90002A4E40F20110C6F800022748001F0560E7
:100BA0003804C6F80403F76005211A20FFF7A6FBF6
:100BB0001A20FFF78DFB1D490839C1F80080081D78
:100BC000066019481949283010390860174A311D44
:100BD0000C3A116015491839086018480C30091D85
:100BE000086000E004E011494FF460705C3908606F
:100BF000657027700020BDE8F0810E20FBE707201C
:100C0000F9E70000280000209C000020A00300203D
:100C10001C150040E743C323A363E313080200202D
:100C200010A5004000A000400011004060F5014008
:100C300040A100400010004008A5014000A0014074
:100C400070B505461E48007880B385B31D4CA06A78
:100C500070B30120FFF731FB606A54F820100A7866
:100C60002A7054F820104978697054F82010897857
:100C7000A97054F820100979297154F82010C97806
:100C8000E97054F82010681D491DFFF7D5FA606A15
:100C9000401C6062082801D300206062A06A401EE8
:100CA000A0620120FFF714FB002070BD01E002E00C
:100CB00003E00820F9E70E20F7E70520F5E700003C
:100CC000280000203003002070B5134E04467078D1
:100CD00008B1112070BDCCB10F483430407C0528DC
:100CE00016D04FF07F452046FFF725FD284204D15E
:100CF0000A48006810F0FF0F0CD0206870630120D4
:100D000000F024FBBDE87040FFF740BD0E2070BD31
:100D1000034DE8E7072070BD28000020241500409F
:100D20000000FFFF70B51F4D0446687808B1112020
:100D300070BD84B31B483430407C05282DD04FF063
:100D40007F462046FFF7F7FC30421BD11649086862
:100D500010F47F4F23D0086810F47F0F1FD008686D
:100D6000000E1CD0091D0868000E18D0086810F489
:100D70007F0F14D0086810F47F4F10D0086810F06F
:100D8000FF0F0CD02068A863022000F0DFFABDE856
:100D90007040FFF7FBBC0E2070BD044ED1E707206A
:100DA00070BD000028000020241500400000FFFF57
:100DB00070B50C461D49497809B1112070BDB0B11C
:100DC000092C31D2194D3435697C052911D04FF0E9
:100DD0007F412CB1164A12680A4201D102781AB337
:100DE000134A121D12680A420BD1012107E00E209E
:100DF00070BD1049EDE7425CB2B1491CC9B2A142D5
:100E0000F9D30146094822463C30FFF715FAC4F1F0
:100E10000801FF202C74C840A874042000F096FA42
:100E2000BDE87040FFF7B2BC072070BD280000206D
:100E30001C1500400000FFFF074810B5407808B1BE
:100E4000112010BD0548806A18B100F0D9F90020C2
:100E500010BD4FF4807010BD28000020DC01002080
:100E60002DE9F041264F0546387840B155B1287834
:100E700068B120280BD8234E317829B109E0082029
:100E8000BDE8F0810E20FBE7F17C884201D9092002
:100E9000F6E71D4CA06A082801D30420F0E7687823
:100EA000082801D30720EBE70120FFF706FA206AA4
:100EB0002522294654F82000FFF7BEF910486A7829
:100EC0002C30815C491C01F003018154206A54F8E4
:100ED0002020401C08281171206201D300202062CC
:100EE000A06A401CA0620120FFF7F2F9707828B9CF
:100EF000307C18B9787808B900F082F90020BFE793
:100F0000280000209C000020DC01002070B541EA90
:100F10004201DDE904564FF0A04441EA830141EA71
:100F2000052104EB800041EA0641C0F8001770BDBE
:100F300001224FF0A043824011B1C3F80825704749
:100F4000C3F80C25704701224FF0A043824011B135
:100F5000C3F808257047C3F80C25704770B5164CC8
:100F6000164AA068C2F80002A06A15490860154B2D
:100F7000091D9889823808601348012140F80C1F28
:100F80000021C0F83411C0F83811104D4FF4E05072
:100F9000286050142D1D2860C2F80C11187810B963
:100FA0006169002088470B49094808600A48E060E9
:100FB0000320607070BD0000280000200010004079
:100FC00040A500409C00002000A0004004F5014026
:100FD0007E030020041500401910000010B50C4CD1
:100FE000606840F00100606000F096F90948806A8E
:100FF00030B11420FFF777F9BDE8104000F000B9D8
:1010000000206070BDE810401420FFF76CB90000AC
:1010100028000020DC0100202DE9F047414A4FF470
:10102000E05010604049D1F80C31DFF80091002702
:101030003F4CB9F80E004E14DFF8F8800125E3B3F9
:101040003D4B1B68CBB365601660D8F8041041F0C7
:101050000101C8F80410D8F82010401A401CC8F844
:10106000240000F059F999F8000088B109F2E22053
:10107000017869B14078410830480068C0B200F09A
:1010800073F828B1D8F8040040F00400C8F8040050
:101090002B48806A50B199F81000012806D014201E
:1010A000FFF721F9BDE8F04700F0AAB888F8017011
:1010B000BDE8F0471420FFF716B9D8F820C0BCF1FE
:1010C000010CC8F820C00BD265601660401CC8F83F
:1010D0002400D8F8040040F00200C8F80400E5E756
:1010E000D8F808000F4640F00802C1F80022D8F8EE
:1010F0001800D8F81410007888471048114928388B
:1011000001601148C8F80C00022088F80100256031
:101110000448001F0660D4F84401002800D03D6058
:10112000BDE8F08708F50140001000409C00002059
:1011300000A0004028000020001400402C150040B2
:10114000DC0100205C0300205D0F00000549002049
:1011500008624862886201F5AA7108624862886282
:1011600070470000DC0100202DE9F041224C0746C9
:101170008846A06A08283DD2A4F5257120460A7841
:101180000026006A01F2E225012A03D04A7842B122
:10119000C97C02E0297820292CD854F8202011702D
:1011A00002E054F820100E7054F82000A91C10F82A
:1011B000052BFFF741F8206A54F820104F700F49B3
:1011C000096854F82020917054F8202082F8048097
:1011D000697854F8202041F30001491C401CD1706B
:1011E0002062082800D32662A06A401CA062012069
:1011F000BDE8F0810020FBE73003002048150040E7
:101200002DE9F05F3E4C4FF00108C4F824803D48C2
:10121000DFF8F4A0A0F5A077416A3C4D4FF0000B39
:1012200050F82110A161387807F5307610B1012807
:1012300044D10DE0087861698847A1690879307068
:1012400086F801B011F8052BB01CFEF7F5FF18E089
:10125000C87828B3387D18B30020814608783070EC
:1012600008794006000E7070CA78DAB10022104387
:10127000707011F8052BB01CFEF7DEFFB9F1000FFE
:1012800012D0A06840F00800C5F800021120C5F88F
:101290000403F88920620220C4F80CA060700DE0FD
:1012A0000120DAE70122E2E7A068C5F80002102079
:1012B000C5F804031648E06084F80180A069154A67
:1012C000417811604078444608FA00F0111D08602A
:1012D0000B48104934302439C07C0860081F066070
:1012E0000120FEF7DFFF0120FEF7F2FFC5F804B191
:1012F000C5F808B1C5F810B12C60BDE8F09F00003A
:1013000028000020DC0100205D0F000000100040DC
:10131000DD0F00002C15004010B50B4CA06A002812
:1013200011D00120FEF7C9FFA06A401EA062606ACA
:10133000401C6062082801D300206062BDE81040B4
:101340000120FEF7C5BF10BDDC01002010B504462A
:10135000C00704D00F48FFF7EEF90F490860A00757
:1013600006D50C48001DFFF7E6F90B49091D08607A
:1013700060070DD507480830FFF755FA06490831D0
:10138000086004480C30FFF74EFA03490C3108603E
:1013900010BD00005C0000201C1500400A48017AC6
:1013A0000A4801600A4849B1012905D0032909D03A
:1013B000042901D000207047302100E040218162E3
:1013C000012070474921FAE79C00002010150040D9
:1013D0002800002070B500F041F8FFF7DFFF194C3E
:1013E000194922787AB1012A0BD000220240607A92
:1013F000B8B1164B1D1F01280ED0022807D00025BA
:1014000013E0134A00E0134A4A610122EEE74FF667
:10141000FF761E60104B03E0FF261E6040F20713AC
:101420002B600A4B083B1860012549691540E07C98
:101430008847A089872801D3012000E000202840A8
:1014400070BD00009C000020280000203C150040DA
:101450009D1400007114000021100100024803498E
:10146000807A0860704700009C0000200C15004046
:10147000084A074911600849497C491E090441EAA4
:101480000021014341F08070111D08607047000089
:1014900000010100141500405C00002007490648C7
:1014A000086007480749407C401E41EA0040034964
:1014B000091D086070470000060003001415004075
:1014C0005C0000202000000100000000000000007F
:1014D0000338FDD870470000010000000000000044
:1014E00001020000FA0003000001022000000000D9
:1014F000111213140D0E0F1018150000000000201B
:1015000074000000180700008C1500007400002013
:101510004C23000028070000080000000001000024
:1015200000110000000000000000000000000000AA
:1015300000000000000000000000000000000000AB
:101540000000010000000000130100000000000086
:10155000000000000000000000000000000000008B
:10156000000000000000000000000000000000007B
:1015700000000000E7E7E7E7C2C2C2C2E7C2C3C497
:0C158000C5C6C7C80805FF020090D003D4
:0400000500000201F4
:00000001FF
